:100000000C94D3010C945D1A0C94F0010C94F00143
:100010000C94F0010C94F0010C94F0010C94F0019C
:100020000C94F0010C94F0010C948A210C945E2243
:100030000C949E1C0C94F0010C94F0010C94F001B3
:100040000C94F0010C94F0010C94F0010C94F0016C
:100050000C94F0010C94411D0C94F0010C94F001EF
:100060000C94F0010C94F0010C94F0010C94F0014C
:100070000C94F0010C94F0010C94F0010C94F0013C
:100080000C94F0010C94F0010C94F0010C94F0012C
:100090000C94F0010C94F0010C94F0010C94F0011C
:1000A0000C94F0010C94F0010C94F00129001E0056
:1000B0001F002000210022002B0014001A0008005D
:1000C00015001700E10004001600070009000A00EF
:1000D00028001D001B00060019000500000000009C
:1000E0002F003000E200225200000000E300E00098
:1000F0002C004C00230024002500260027002A00A5
:100100001C0018000C00120013004C000B000D0026
:100110000E000F00330034001100100036003700CD
:10012000380031002152E6002D002E0000000000B2
:1001300053002C00E400E7000000000035021E021E
:100140001F02200221022202010001000100010021
:1001500001002F0001004A004B004E004D00260216
:100160000100010001000100010001000000000089
:100170000100460001000100000000000100010034
:1001800001000100230224022502260227024C005E
:1001900030005F006000610001002E0227025C0059
:1001A0005D005E002D003102010059005A005B0025
:1001B0002E002D020100010001006200000000007D
:1001C00001000100010001000000000045003A00AC
:1001D0003B003C003D003E00010001000100010029
:1001E00001002F0001005000520051004F00260274
:1001F00001000100010001000100010000000000F9
:1002000001000100010001000000000001000100E8
:10021000010001003F004000410042004300440053
:1002200030000100530049004700A8002702AC003D
:10023000AE00AB000100A9000100010001000100B7
:100240000100AA00010001002E00010000000000D2
:100250000100010001000100000000002C03440027
:1002600061006300740079006C002D004D00610096
:100270006E00750066006F0072006D00200028009F
:10028000350078003600290000000E03740073006A
:1002900068006F0072007400000004030904090282
:1002A0003B00020100A0FA09040000010301010063
:1002B0000921110100012240000705810308000106
:1002C00009040100010300000009211101000122BD
:1002D0007B000705820320000112010002000000DC
:1002E000084D44363501000102000105010902A153
:1002F0000185020901A10005091901290815002538
:100300000195087501810205010930093115812522
:100310007F95027508810609381581257F9501753D
:10032000088106050C0A38021581257F950175089C
:100330008106C0C005010980A101850319012AB702
:1003400000150126B700950175108100C0050C0944
:1003500001A101850419012AA002150126A0029518
:100360000175108100C005010906A101050719E00A
:1003700029E7150025019508750181029501750889
:1003800081010507190029FF150026FF0095067554
:100390000881000508190129059505750191029547
:1003A0000175039101C011241FBECFEFDAE0DEBF5B
:1003B000CDBF11E0A0E0B1E0EAE4FAE402C00590AC
:1003C0000D92AA3AB107D9F722E0AAEAB1E001C03A
:1003D0001D92A73CB207E1F70E941B140C94E42481
:1003E0000C9400008330B8F46C30A8F4463098F4D4
:1003F00050E096E0699F400D511D1124FA0198E4E8
:10040000899FE00DF11D1124EE0FFF1FE455FF4FF2
:1004100085919491089581E090E008950E94F20101
:10042000089581E008950E941102089581E00895E1
:100430000E94110208950E941802089508950E94D2
:100440001E020895A6E0B0E0E8E2F2E00C94402439
:1004500049835A839E833091B10189819A813111F8
:100460001AC03E81332399F0222389F00E94230889
:10047000182F682F89819A810E94FF0769817A81EC
:10048000812F0E94150F2696E3E00C945C240E94B5
:100490001108182FF3CF0E94230869817A81F1CFC8
:1004A000FC01262F40815181628173818481958175
:1004B0000E9422020895CF93DF93EC0161E00E9435
:1004C0005002BE010E941302DF91CF910895CF9395
:1004D000DF93EC0160E00E945002BE010E941F0207
:1004E000DF91CF91089508950E94D4060E9473026F
:1004F0002FEF84E39CE0215080409040E1F700C062
:10050000000008950E9474020E94651D08950E94D3
:1005100074020E94761D08950F931F93CF93DF936B
:100520008C0161E00E945002EC01B8010E941B02A4
:10053000811106C080E0DF91CF911F910F91089546
:10054000B801CE010E947B198823A1F3B801CE0126
:100550000E94C416882371F3B801CE010E94ED18E1
:10056000882341F3F8018581882361F0C330FCE7DB
:10057000DF07E9F058F4C115ECE7DE07A9F0C13058
:10058000DC47B9F0C8010E941602D5CFCB358CE705
:10059000D807A9F0CC35ECE7DE0771F0CA35DC47A7
:1005A00089F70E946A0CEECF0E948202C3CF0E949C
:1005B000720C0E948702BECF0E94600CE3CF0E94A3
:1005C0006E0CE0CF0E947B1C0E94090308950E94DC
:1005D0000D030E94801C0895089581E008950895F8
:1005E000CF93DF93D82F0E94ED02C82F882319F0F4
:1005F0008D2F0E94EF028C2FDF91CF9108950895E7
:10060000CF93C82F0E94EC028C2F0E94F002CF9152
:10061000089580E00E94000308950E94831B0E94B9
:1006200000030895CF930E94831BC82F8091AC01D3
:100630008C1779F0C093AC010E940A1D6093AD0144
:100640007093AE018093AF019093B0018C2F0E9404
:100650000003CF910895ADE0B0E0E1E3F3E00C9446
:100660004124488759876A877B878C879D879111AA
:100670000E94980B1F8286E0FE013896DE011196DB
:1006800001900D928A95E1F78D8181110DC029812C
:100690003A814B815C816D817E818F810E94CB0A82
:1006A0002D96E2E00C945D24CE0101960E945B023F
:1006B0008111EDCFF5CFFC012481213021F480811F
:1006C00091810E9455080895662329F00E949F1485
:1006D0000E94721508950E94F914FACFCF93C82F83
:1006E0008823C9F08238C9F40E94831B81FD13C09E
:1006F00089E30E94500B0E94D10B2FEF87EE93E00D
:10070000215080409040E1F700C0000089E30E9442
:10071000580B0E94D10BCF9108958338A1F40E9409
:10072000831B80FDF8CF83E50E94500B0E94D10B04
:100730002FEF81EE94E0215080409040E1F700C01F
:10074000000083E5E4CF8438A1F40E94831B82FD7E
:10075000E2CF87E40E94500B0E94D10B2FEF81EE75
:1007600094E0215080409040E1F700C0000087E411
:10077000CECF8CEF8C0F813AB8F48C2F0E943118B9
:100780008111C9CF6C2F80910001909101010E94CD
:100790000C1C882329F08C2F0E94580B0E94D10B2F
:1007A0008C2F0E94500BB5CF80E28C0F883048F41C
:1007B000C77081E001C0880FCA95EAF70E947B0BE1
:1007C000A8CFEBE5EC0FE33040F4F0E0E05AFE4F49
:1007D000808190E00E94B01B9ECFE8E5EC0FEB31EA
:1007E00050F4F0E0EE0FFF1FE65DFE4F8081918137
:1007F0000E94D51B90CF83E38C0F833108F08BCF01
:1008000061E08C2F0E94640386CF882309F456C0D0
:10081000823879F40E94831B81FF50C089E30E94D3
:10082000500B0E94D10B89E30E94580B0E94D10B00
:100830000895833859F40E94831B80FF3FC083E5ED
:100840000E94500B0E94D10B83E5EECF843859F4FF
:100850000E94831B82FF32C087E40E94500B0E94DB
:10086000D10B87E4E1CF9CEF980F913AE8F290E248
:10087000980F983050F4877091E001C0990F8A95D5
:10088000EAF7892F0E94810BD1CF9BE5980F933017
:1008900028F490E080E00E94B01B089598E5980F3E
:1008A0009B3128F490E080E00E94D51B089593E3EB
:1008B000980F933118F460E00E94640308951F9329
:1008C000CF93DF93182FEB010E946E03209739F42A
:1008D000812F0E940504DF91CF911F9108958FE928
:1008E0009FE00197F1F700C000002197EFCF70E083
:1008F00060E0893311F460E570E00E945F040895C0
:10090000882321F00E947B0B0E94D10B089588233D
:1009100021F00E94810B0E94D10B0895B0E0A0E06D
:10092000E4E9F4E00C943A246C01D62FC72FFC01C3
:100930001581068102950F700E94710BE82E8823A5
:10094000E9F0E12E1123D1F08C2F807F803451F01B
:1009500080E28D0F8830F8F0011104C08C2F807E6A
:100960008032C9F080919B0282FF15C082E00E9414
:10097000340C0E94710B91E0E82EE926BC2EB29453
:100980009FE0B922FBE0FB15B8F1EB2DF0E0EA5156
:10099000FB4D0C942B24E12CF1CF0C2F0F70C07F5A
:1009A00011F00295007F112399F0002359F080E2A5
:1009B0008D0F883010F0D11107C0802F0E947B0B63
:1009C0000E94D10B8D2F5AC0802F0E948B0BF8CF25
:1009D0008D2F0E940504002379F080E28D0F88306E
:1009E00010F0D11104C0802F0E94810B03C0802F12
:1009F0000E94910B0E94D10BEB2DE850FF0B349716
:100A000020F40E94831B0E940003EE2089F00E94C4
:100A10006D0B80FD0DC0F60115820E94670B0E94D0
:100A20005D07C6010E949B060E94670B0E946D072E
:100A3000CDB7DEB7E9E00C9456242C2F2F70F22EA0
:100A4000C07FC03219F0F29480EFF822DD2341F02C
:100A5000D130D1F1112309F444C00023F1F0B2CF19
:100A600080919B0282FD15C0112359F0FF2029F0CF
:100A70008F2D0E947B0B0E94D10B80E00E946E03A1
:100A8000BBCF80E00E940504FF2009F4B5CF8F2D75
:100A9000ABCF112369F0011104C08F2D0E94800497
:100AA000ABCF013009F0A8CF8F2D0E94AF0BA4CFA0
:100AB0000111A2CF8F2D0E9487048F2D0E94BB0BA6
:100AC0008F2D0E949F0B98CF112321F0063008F044
:100AD00093CFE3CF053008F08FCF8F2D0E9487048E
:100AE0008BCF0023D1F3D93349F43FEF87EE93E066
:100AF000315080409040E1F700C000008D2F0E94EF
:100B000005047ACF8C2F86958695837069F08130A5
:100B100009F072CF8D2F9C2F9370111102C080E0CD
:100B200090E00E94D51B68CF8D2F9C2F93701111E0
:100B300002C080E090E00E94B01B5ECF612F8D2F3D
:100B40000E94640359CF8C2F8370A1F5111154CFEB
:100B50004D2F429546954770440F440F2D2F2F700F
:100B600030E0042E02C0220F331F0A94E2F790E017
:100B700080E0D4FF09C08FE090E002C0880F991F89
:100B80004A95E2F780959095C695C695C370822BDD
:100B9000932BC23049F058F4C13019F00E942D0750
:100BA0002BCF0E94240728CF0E94360725CF0E9412
:100BB000210722CF8695112311F08C2F8170882375
:100BC00009F41ACF4D2F429546954770440F440FB4
:100BD0002D2F2F7030E0042E02C0220F331F0A94F5
:100BE000E2F790E080E0D4FF09C08FE090E002C01F
:100BF000880F991F4A95E2F780959095C695C695FE
:100C0000C370822B932BC23049F058F4C13019F0D5
:100C10000E949807F1CE0E948F07EECE0E94A10796
:100C2000EBCE0E944507E8CECF70112329F08C2F20
:100C30000E945D078D2F32CF8D2F0E9487048C2F4D
:100C40000E946D07D9CED23F41F160F4D03FB9F098
:100C5000D13F81F0112309F446C00111B3CE8C2F8E
:100C60008F711FC0D33F01F1D43FA1F780919B0248
:100C700082FD24C08C2F8F71112311F312C0112318
:100C800041F0053008F0B8CE8C2F8F710E947F079D
:100C9000B3CE063008F0B0CEF7CF8C2F8F71111184
:100CA000CFCF0E945D07A8CE112329F08C2F8F7122
:100CB0000E945107A1CE0E944C079ECE112349F0FD
:100CC000CF718C2F0E945D0763E08C2F0E94160C61
:100CD00093CE81E00E94340C023008F48DCE82E085
:100CE0000E94340C89CE002359F0D93309F006CF85
:100CF000EFEFF7EE23E0E150F0402040E1F7FCCECB
:100D00008C2F8F719DCF0F931F93CF93DF93EC01A7
:100D1000688179818D810E9460088C010E94AA07F8
:100D20000E942007B801CE010E948E04DF91CF916E
:100D30001F910F910895CF93DF93EC018C8188234D
:100D400099F0CE010E948C02811111C00E94710B9A
:100D5000882351F08D81882339F080919B0282FF96
:100D600003C082E00E94340CDF91CF910895CE0140
:100D70000E948306CE010E946702F6CF90E080E0D9
:100D80000E94B01B90E080E00E94D51B0E94980B4F
:100D90000E94D10B0E948E150E94721508950E9428
:100DA000600B0E94BE0608950E94880B0E94CF0629
:100DB000089592959F70963091F058F4925F9F70CD
:100DC000923058F4803F19F030F4883E30F481E0DE
:100DD00008959A5FF4CF843FD1F380E00895883E70
:100DE000B0F3813FD1F7F3CFFC012481222339F006
:100DF000808191810E9455080E94D906089580E063
:100E00000895A6E0B0E0E7E0F7E00C9441242696D0
:100E1000E2E00C945D24A7E0B0E0E1E1F7E00C949F
:100E200041242796E2E00C945D2408950E94150762
:100E300008950E9416079093D9018093D8010895D0
:100E400008950E94190708952091D8013091D90181
:100E5000822B932B0E94190708952091D80130917D
:100E6000D901822393230E94190708952091D80164
:100E70003091D901822793270E94190708950E9473
:100E8000150708950E943F0708950E944207909316
:100E9000D7018093D601089590E080E00E94450735
:100EA000089521E030E0A90102C0440F551F8A9542
:100EB000E2F7CA010E944507089521E030E002C030
:100EC000220F331F8A95E2F78091D6019091D701C6
:100ED000822B932B0E944507089521E030E002C049
:100EE000220F331F8A95E2F7209530958091D60125
:100EF0009091D701822393230E944507089521E012
:100F000030E002C0220F331F8A95E2F78091D601AC
:100F10009091D701822793270E9445070895209139
:100F2000D6013091D701822B932B0E94450708955B
:100F30002091D6013091D701822393230E94450747
:100F400008952091D6013091D701822793270E94DE
:100F5000450708950895262F277091E001C0990F45
:100F60002A95EAF723E0769567952A95E1F7660FCB
:100F7000771F660F771FFA01E60FF71F50E040E07A
:100F8000682F70E08191DF0111979B01042E02C050
:100F9000369527950A94E2F7217021952827292371
:100FA00028272C934F5F5F4F4430510559F7089520
:100FB000A82FA77023E0969587952A95E1F7880FCB
:100FC000991F880F991FFB01E80FF91F50E040E0BF
:100FD00080E0219130E00A2E02C0369527950A94D0
:100FE000E2F721703327042E01C0220F0A94EAF79A
:100FF000822B4F5F5F4F4430510559F70895262FDC
:101000009C3070F4863060F4682F70E086E0989F22
:10101000600D711D112442EB51E0822F0E94AB073D
:101020000895292F9C3068F4863058F490E062EBE4
:1010300071E036E0239F800D911D11240E94D80796
:10104000089580E00895B0E0A0E0E9E2F8E00C94B3
:101050003A247C010091D6011091D7018091D801EA
:101060009091D901082B192BCFE0D0E0CC24C39468
:10107000D12CBC2EC6010C2E02C0880F991F0A94D9
:10108000E2F780239123892B49F4219790F7B12C23
:101090008B2DCDB7DEB7E9E00C945624B7018C2F29
:1010A0000E94210F019789F3F3CFCF93DF93EC01D7
:1010B0000E942308BE010E94210FDF91CF91089565
:1010C0001F93CF93DF93EB019091B101992339F0F6
:1010D000CB010E945508DF91CF911F91089588237D
:1010E00069F0CB010E942308182F682FCE010E94BF
:1010F000FF07BE01812F0E94210FEDCFCB010E947F
:101100001108182FF6CF1F93CF93DF93C091DA0108
:1011100017E08091DB018C1304C0DF91CF911F9108
:101120000895D0E01C9FF0011D9FF00D1124E452A2
:10113000FE4F208131814281538164817581868196
:101140000E940B072196C770E4CF209114023091C2
:101150001502409116025091170260911802709189
:10116000190280911A020E940B070895CF93DF9312
:1011700080911A02807F09F04DC080911902882366
:1011800009F448C0E091DA015091DB01C0911502E9
:10119000D0911402609116027091170247E05E1719
:1011A000C9F18E2F90E0E49FF0011124E452FE4F2C
:1011B0002481222391F1489FF001499FF00D1124D1
:1011C000DF01A452BE4F11962C9111972C1325C00C
:1011D0002C912D1322C015962C91159721111DC00D
:1011E00012962D913C91261B370B283C3105A8F413
:1011F00080911A028F70806180931A02EE51FE4F27
:1012000080818F708061808384E192E00E949B06E0
:101210000E948308DF91CF910895FC013196E77019
:10122000BECF482F2091DA019091DB0157E02913BE
:1012300002C080E0089530E0529FF001539FF00D0E
:101240001124E452FE4F8181681306C08081481347
:1012500003C085818111EECF2F5F3F4F2770E7CF0D
:10126000A4E1B0E0E6E3F9E00C9437248C0186E0D9
:10127000F801DE011F9601900D928A95E1F7D801E1
:1012800014968C9114971596EC90159794E1A92ECD
:1012900092E0B92E9091180291111FC08823D1F0CD
:1012A000EE20A9F0C8010E94F406F82E882379F0F8
:1012B00087E0F801D50101900D928A95E1F7C5010B
:1012C0000E945B030E94B6080E94A5083DC0C801A9
:1012D0000E949B06FF24F39437C0F801C080D180A0
:1012E00082809380F09019022091160230911702AB
:1012F000A401421B530BFF2009F4F6C0483C5105E2
:1013000008F0A5C0882301F19091150280911A027E
:10131000282F207F09F067C0D9121BC090911402BA
:101320009C1117C0E11059C08F70806180931A0220
:101330000E94A50884E192E00E949B0680911A0217
:10134000D80116968C93F12C8F2D6496ECE00C94BA
:101350005324E11042C06D2D8C2D0E941109E82EFE
:10136000882371F084E192E00E949B0687E0E4E12B
:10137000F2E0DF011D928A95E9F70E94A508E3CF0C
:10138000CF86D88A8F8598890E945508292F229563
:101390002F70243058F49F70223088F0992399F0F0
:1013A000F8019681907F79F4FE2CCECF2A5F2F70C2
:1013B000223068F0C8010E949B06EF2CF5CF9923DC
:1013C00011F0882389F3805E883070F3F3CF803F7B
:1013D00058F3815F833070F7E7CF80911A02816004
:1013E00080931A02B0CFD91207C0909114029C11B9
:1013F00003C0EE2009F49CC0C8010E94F4068823B3
:1014000009F465CFEE2009F462CF80911A02803290
:1014100088F02091140230911502398728879B8625
:101420008A86909118029C871D868E87CE01089629
:101430000E949B0687E0F801A4E1B2E001900D92C2
:101440008A95E1F70E94B6080E94A50843CF9091C3
:101450001A02292F207F91F4682D9A8A898AA60181
:101460007A899E2D0E94010784E192E00E949B06EA
:1014700087E0F50111928A95E9F77FCF882309F477
:1014800063CF809115028D1111C0809114028C11CF
:101490000DC0E1100BC016969C93C8010E949B06DC
:1014A00087E0F50111928A95E9F74ECFC8010E94B5
:1014B000F406882309F40BCFEE2009F408CF8091BD
:1014C0001A02803208F4B6CF20911402309115022E
:1014D0003A8329839C828B82909118029D831E827D
:1014E0008F83CE010196A4CF483C510508F045C03A
:1014F000882309F4EFCEFE2CEE2009F4E8CE80918B
:1015000015028D112CC0809114028C1128C080917D
:101510001A0280FD1BC0982F907FC1F016968C9305
:101520001697903F39F0982F907F905F8F70892B9E
:1015300016968C93C8010E949B0687E0F801A4E1EF
:10154000B2E001900D928A95E1F7BECE87E0F801F6
:10155000A4E1B2E001900D928A95E1F7F5CEC801C1
:101560000E94F406811166CF80911A0281608093F7
:101570001A02C8010E949B06E7CE682D9A8A898AC2
:10158000A6017A899E2D0E94010787E0F50111923C
:101590008A95E9F799CEAEE0B0E0E1EDFAE00C947F
:1015A0004024288739874A875B876C877D878E87A9
:1015B000CE0108960E9430098823B1F06C8566231D
:1015C00041F0288539854A855B857D858E850E9419
:1015D0000B0717E08091DA019091DB0189133DC080
:1015E0002E96E3E00C945C2487E0FE013896DE0141
:1015F000119601900D928A95E1F78C85882349F325
:101600002091DB0130E0C901019687709927409154
:10161000DA014817190699F097E0929FD001939F3D
:10162000B00D1124A452BE4FFE01319601900D92CF
:101630009A95E1F78093DB010E948308CACF0E944C
:10164000D4061092DB011092DA0187E0E4E1F2E0C7
:10165000DF011D928A95E9F7BCCF819FC00111245B
:1016600084529E4F0E943009882309F4B9CFE0913B
:10167000DA011E9FF0011124E452FE4F20813181D6
:10168000428153816481758186810E940B0780911C
:10169000DA0190E00196877099278093DA019ACF5A
:1016A000682F80910001909101010E94421C0895D1
:1016B000682F80910001909101010E94451C0895BE
:1016C00080910001909101010E94481C0895809131
:1016D00023028695869586950895809123028770CA
:1016E000089590912302977081E009F480E00895B5
:1016F00080912F02089590912F02892B80932F02C1
:101700000895809590912F02982390932F02089529
:1017100010922F02089590912E02892B80932E0211
:101720000895809590912E02982390932E0208950B
:1017300010922E02089508950E949B0B0895909197
:101740002402292F282331F08095892380932402B5
:101750000E949C0B089508950E94AB0B08959091F0
:101760002502292F2823281729F0982B909325024A
:101770000E94AC0B089590912502292F282331F067
:1017800080958923809325020E94AC0B0895809157
:101790002502882329F01092250280E00E94AC0BDC
:1017A0000895CF93DF93E0910001F09101018091C2
:1017B0002F028083E0910001F091010180819091DE
:1017C0002E02892B808390912502992381F0E0914C
:1017D0000001F09101018081892B808380910001BB
:1017E000909101010E94FA1B81110E94C70BC091C8
:1017F0000001D091010148E050E06BE172E0CE01C0
:101800000E947C24892B59F088E0FE01ABE1B2E014
:1018100001900D928A95E1F7CE010E94971BDF910E
:10182000CF91089508950E94120C089590919B0203
:1018300092FF11C098E0899F90011124622B609360
:1018400023020E945D0780912302869586958695E6
:101850000E94130C08950E945D07089510922302C0
:1018600080E00E94130C08959091230280958923B3
:1018700080932302282F277069F4891759F09091DB
:101880009B0292FF07C08695869586950E946D07FC
:101890000E942E0C089590919B0292FB222720F922
:1018A000281769F080FB92F990939B0280919A022D
:1018B00090919B020E94930C82E00E94340C089548
:1018C00080919B0282FB882780F991E089270E9402
:1018D0004B0C089581E00E944B0C089580E00E941B
:1018E0004B0C08956FEF7FEF90E080E00E94CE24D4
:1018F000089590E080E00E949A2421E0863E9E4F69
:1019000009F020E0822F089582E090E00E94922466
:10191000089583E090E00E949224089584E090E08E
:101920000E949A240895BC0184E090E00E94CE2495
:101930000895AB01BC018FE090E00E94C22408959D
:10194000AB01BC0183E190E00E94C224089560E0F5
:1019500070E0CB010E94A00C089560E070E0CB0124
:101960000E94990C0E94A70C0895A8E0B0E0EBEB50
:10197000FCE00C94412466EE7EEF90E080E00E9453
:10198000CE2460E082E090E00E94B02460E083E03A
:1019900090E00E94B0241092D9011092D80160E02A
:1019A00074E184E090E00E94CE2460E086E090E064
:1019B0000E94B0246FEF87E090E00E94B02440E0E6
:1019C00050E0BA0188E090E00E94C22460E084E226
:1019D00090E00E94B02460E087E190E00E94B02493
:1019E00060E08CE090E00E94B02460E08DE090E048
:1019F0000E94B02419821A821B821C821D821E82C0
:101A00001F82188648E050E068E170E0CE01019640
:101A10000E94A02440E050E0BA0180E290E00E94E1
:101A2000C2240E94AD0C2896E2E00C945D240E9432
:101A3000B50C0895682F8EE090E00E94B0240895C0
:101A4000A6E0B0E0E6E2FDE00C943F240E94FE1C1C
:101A50008C0180913002909131028017910781F0C2
:101A600019821A820E94FE1C682F49815A81792F9F
:101A700080E090E00E942B0310933102009330022B
:101A80002696E4E00C945B240E943110609342029D
:101A900070934302809344029093450260933E0208
:101AA00070933F02809340029093410208950895FD
:101AB00008950E94580D089508950E945C0D0895A0
:101AC00081E008958BE490E10E94791B0E94570DFC
:101AD0000E94590D08950E941712089508950895BF
:101AE0000E946E0D0E946F0D08950E944E100E947C
:101AF000FF0208950E94F51C0E940B100E943212F2
:101B00000E9478110E94750D0E94AC160E943C1232
:101B10000E945D0D0895A6E0B0E0E1E9FDE00C94BF
:101B200038240E94600D81110CC00E94200D0E947B
:101B300017120E94B0150E9412032696EBE00C9437
:101B400054240E949B1182E3A82E82E0B82E7501D6
:101B500010E0F70101917F01812F0E9474101F5F37
:101B60001C3009F441C00817A1F38091460281FDA1
:101B70000E947A100E946B0DC82E10E09924939455
:101B8000812F0E947410082FF50181915F010817C1
:101B900029F1F12CEE24E394D02ED8268D2D8E2120
:101BA000A9F0CC2099F0F9821A830E94FE1C9C8334
:101BB0008B839D8291E0802F8E2109F490E04981F2
:101BC0005A816B817C818D810E942B03F394EE0CF2
:101BD000F6E0FF12E3CFF501319700831F5F1C3061
:101BE00079F60E94440DA3CF0813BFCF9ECF1F9359
:101BF000CF93DF930E94260FEC01C11580E5D80733
:101C0000F0F5C11580E4D80708F09CC0C03ED105AE
:101C100020F5CD3CD10508F082C0C83AD10578F452
:101C2000C53AD10508F073C0C130D10519F120972C
:101C300009F1C430D105F0F4D0E0C0E01BC0C33CD2
:101C4000D105D0F7C85AD0E0CC0FDD1FCD59DE4FFB
:101C50000990D881C02DD4640DC0C11580E2D80789
:101C600008F0D1C0C11581E0D80708F05AC0C83EBD
:101C7000D10510F7CE01DF91CF911F910895C036A5
:101C800082E5D80718F5C03482E5D80708F06BC0A4
:101C9000C03282E5D80708F05FC0C11582E5D807D9
:101CA00008F497C02C2F2695269580E2289F900156
:101CB00011248C2F8370C1E0D0E002C0CC0FDD1F57
:101CC0008A95E2F7C22BD32BDD68D4CFC03A82E5E8
:101CD000D80760F4C03882E5D80708F459C0CF713E
:101CE000D0E0DC2FCC27C46FD06AC4CFC03C82E5E3
:101CF000D80708F462C0C03E82E5D80708F09CCF40
:101D0000DC2FCC27CC27DF71C06FD06AB3CFC55A88
:101D1000D0E0C756DE4FC881D0E0D064ABCFD065ED
:101D2000A9CF8D2F0E94C80F182FCE0199270E948E
:101D3000260FC12FD0E0DC2FCC27CC27DF71C82B9A
:101D4000D92B98CFCE0199270E94260FCC27DF7080
:101D5000C82BD92BD06A8ECFCF71D0E0DC2FCC2707
:101D6000C16FD06A87CF2C2F26952695277080E2E9
:101D7000289F900111248C2F8370C1E0D0E002C015
:101D8000CC0FDD1F8A95E2F7C22BD32BDC6872CF14
:101D90002C2F26952695277080E2289F90011124EC
:101DA0008C2F8370C1E0D0E002C0CC0FDD1F8A957C
:101DB000E2F7C22BD32BDA685DCF8C2F8F710E9494
:101DC000C80FC82FD0E0DC2FCC27CC27DF71D06222
:101DD00051CF8C2F8F710E94C80F55E0D695C795B3
:101DE0005A95E1F7CF70D0E0DC2FCC27282F30E0D8
:101DF00084FF05C044E0220F331F4A95E1F7C22B50
:101E0000D32BD06937CF8D2F8F710E94C80F182F19
:101E1000CE0199270E94260FC12FD0E0DC2FCC27BE
:101E2000CC27DF71C82BD92BD2CF462F7C3030F492
:101E3000663020F4672F0E940E02089590E080E043
:101E400008950E94150F0E94F70D0895823891059C
:101E5000B9F1B0F48133910509F47DC048F48932B9
:101E6000910509F46DC08A32910509F47BC008958B
:101E70008533910509F45FC08933910509F108950F
:101E8000833E9105D9F138F4803E910529F1823ED7
:101E9000910579F10895863E9105D9F1873E910526
:101EA00009F43EC0843E910541F520919B0221FF3B
:101EB00024C080919A0284FD19C087EE90E00895B5
:101EC00020919A02237009F05AC020919B0223FFAF
:101ED00014C089E290E0089520919A0220FD38C054
:101EE00030919B0230FF09C024FF43C090E080E0A6
:101EF000089520919A0222FDF7CF089520919A0229
:101F000022FD3AC030919B0230FD39C024FFF5CF4D
:101F1000EDCF20919A0223FFF0CF24FDE7CFCDCF64
:101F200020919A0223FD2EC030919B0231FFEECF0B
:101F300084EE90E0089520919A0225FFDECFC9CF6C
:101F400020919A0225FD21C020919B0223FFD5CF2D
:101F500089E390E0D2CF20919A0226FFCECF8AE289
:101F600090E0089520919A0226FFC7CF81E390E088
:101F7000089583EE90E0089582EE90E0089580EE5B
:101F800090E0089586EE90E0089585E390E008954E
:101F900090919A0292FF06C0282F28712830F9F4F8
:101FA000877F846093FF06C0282F28712831F1F4C1
:101FB000877E846120919B0220FF06C0382F3871F4
:101FC0003830D9F4877F816021FF06C0282F28711F
:101FD0002831D1F4877E816194FD877E0895282F72
:101FE00024712430F9F68B7F8860DCCF282F247190
:101FF000243101F78B7E8861DDCF382F317131308C
:1020000019F78E7F8860E0CF282F2171213121F7C9
:102010008E7E8861E1CF1092960210929702109204
:102020009802109299020895CF92DF92EF92FF9258
:102030006B017C010E94171281110EC00E940A1DC3
:10204000C61AD70AE80AF90AC0929602D0929702F5
:10205000E0929802F0929902FF90EF90DF90CF907B
:1020600008950F931F930E941712882329F00E944E
:102070000A1D1F910F9108950E940A1D009196025A
:10208000109197022091980230919902600F711F70
:10209000821F931FEECF80E0089508950E94790C6F
:1020A000811102C00E94170D0E94840C8093460289
:1020B0000E948E0C90939B0280939A020E944D1076
:1020C0000E94890C90E00E9421078091D601909196
:1020D000D7010E944207089508950E946C10089548
:1020E00008950E9470100895E82FF0E0E755FD4F25
:1020F00080810895089580EA8A95F1F7089500C0D7
:1021000008950E947B10089508950E9484100895F8
:10211000A6E0B0E0EEE8F0E10C943D240E94171236
:10212000F82E6091B502882309F440C086E0E82EBD
:102130008E010F5F1F4FF8018E2D11928A95E9F7DE
:10214000862F90E0B80187559D4F0E944A12882340
:10215000B9F080919C0290E046E050E0B8018755CC
:102160009D4F0E947C2421E020934702892B91F40B
:10217000F12C0E9471108F2D2696E6E00C945924C4
:10218000809147028823A1F3F8011192EA94E9F7BC
:1021900010924702A0919C02B0E0A755BD4F86E087
:1021A000F80101900D928A95E1F7E3CF70E0675551
:1021B0007D4F80919C0290E087559D4F0E94D112E7
:1021C0000E948510D8CFF894E82FE295EF70F0E0E8
:1021D00031A1282F2F7081E090E001C0880F2A954F
:1021E000EAF7982F9095932391A392A1892B82A32C
:1021F000789408950F931F93CF93DF93C2EAD1E0B1
:1022000089918F3F11F00E94E31081E0C83AD8070E
:10221000B9F7CCE9D1E002EA11E089918F3F11F0E2
:102220000E94E3100C171D07C1F7DF91CF911F919A
:102230000F910895B0E0A0E0E0E2F1E10C943B24BE
:10224000EC01D62E062F10E0C8018E559E4F7C0162
:10225000FC0180818F3F09F444C0F894E82FE29597
:10226000EF70F0E091A18F7021E030E001C0220F0B
:102270008A95EAF7892F822B81A382A120952823B2
:1022800022A378940E947F10ECE9F1E031E0C12CA8
:1022900021912F3F59F1A22FA295AF70B0E09096F7
:1022A0008C9190E02F7002C0959587952A95E2F762
:1022B00080FD1CC0832FC82A330F81E0E23AF80763
:1022C00039F7F70180818F3F11F00E94E31061E040
:1022D000C11001C060E08D2D0E948110C00FD11F80
:1022E000C882CDB7DEB7E8E00C94572480E0E3CF96
:1022F000809102018091020196E0811190E090931B
:10230000B50286E0891B80939C020E94FA108CE043
:10231000E9EAF2E0DF01982F1D929A95E9F7EDE9DD
:10232000F2E0DF011D928A95E9F786E00E94D9115B
:102330000E946D100895ACE0B0E0E1EAF1E10C9488
:102340003E248E010F5F1F4F8CE0F80111928A9599
:10235000E9F7F12C6F2DC8010E941A11F394F6E0F1
:10236000FF12F8CF4CE050E0B8018DE992E00E94F6
:102370007C2421E0009709F420E0892B41F08CE0D7
:10238000F801ADE9B2E001900D928A95E1F7609114
:10239000B50270E067557D4F46E08DE992E00E94FE
:1023A000DA11182F0E948810812B2C96E5E00C94EE
:1023B0005A240895CF92DF92EF92FF920F931F93CA
:1023C000CF936C017B01042F222349F081E080939D
:1023D0004A020E94FE1C9093490280934802C091D9
:1023E0004A02C1110AC0C0E08C2FCF911F910F91FA
:1023F000FF90EF90DF90CF900895809148029091E8
:1024000049020E94161D059770F310E0A801B6015D
:10241000C7010E947C24892B41F0A801B601C701A5
:102420000E94892410924A02DFCFC0E0FBCF809146
:102430004D02811107C00E940A24882351F081E0D7
:1024400080934D0281E090914D02913009F080E03F
:10245000089582E080934D020E940524F3CF0E94EC
:10246000171208950E942F12809302010E941712E2
:1024700081110E94801208950E941712811102C0DA
:102480000E948312089581E090914E029A3008F0E4
:1024900080E008950F931F93CF93DF93EC018B019E
:1024A00080914E028A30B8F4B801CE010E94CE125B
:1024B000C82F811122C080914E028F3FB9F40E9433
:1024C000FE1C90934C0280934B028C2FDF91CF9196
:1024D0001F910F91089580914B0290914C020E94A0
:1024E000161D843F914000F7C0E0EFCF8F5F8093CF
:1024F0004E028A3020F7C1E0E8CF10924E02E5CFBD
:102500000E94171A08950E941A1A0895B0E0A0E0D8
:10251000ECE8F2E10C943C247901C82F880FDD0B24
:1025200041155105A9F0FE0193E0EE0FFF1F9A95AA
:10253000E1F7ED5FFE4F81819281815B9D4F2081AC
:1025400030E04217530708F49A01A9010E94892438
:10255000CE010E94031BD82E8823D1F0011511054E
:10256000B9F083E0CC0FDD1F8A95E1F7FE01ED5F46
:10257000FE4F438150E00417150708F4A801CD5F12
:10258000DE4F6C817D81615B7D4FC7010E94892494
:102590008D2DCDB7DEB7E7E00C9458240E94C01310
:1025A00008950E94D7130895A4E0B0E0EAEDF2E1A7
:1025B0000C943F24609168027091690280916A02D4
:1025C00090916B020E94251D11E064367105810512
:1025D000910518F10E9431106E5F7F4F8F4F9F4F12
:1025E00069837A838B839C8310E000E030E020E0F5
:1025F00044E050E0BE016F5F7F4F82E00E94861290
:10260000182F882351F00E940A1D6093680270936E
:10261000690280936A0290936B02812F2496E4E012
:102620000C945B24B0E0A0E0E8E1F3E10C943924E1
:102630007C015B016A010E94431201E010E08823E3
:1026400011F00AE010E0C1E0D0E0B501C701F601E9
:102650000995811104C021960C171D072CF4CDB7E4
:10266000DEB7EAE00C945524CC9F9001CD9F300D4D
:10267000300D112490E080E045E34A95F1F7000029
:10268000019682179307C1F7E0CFA7E0B0E0EBE433
:10269000F3E10C9439247B01C090A801D090A901EA
:1026A00001E010E09E01295F3F4F50E040E070E004
:1026B00060E080E00E948612182F882309F448C049
:1026C00056018FEFA81AB80A6091640270916502F2
:1026D00080916602909167020E94251D6436710503
:1026E0008105910568F106E010E09E012F5F3F4FE4
:1026F00050E040E070E060E081E00E948612D82E59
:1027000066E070E0C5010E94AD1611E09F8198134C
:1027100010E01D2141F10E940A1D60936402709334
:102720006502809366029093670286E0FE0131960F
:10273000AEE5B2E001900D928A95E1F711E013C089
:1027400066E070E0C5010E94AD169F818913CBCF72
:1027500086E0F6013196DE01119601900D928A9580
:10276000E1F71111E2CF86E0EEE5F2E0D70101904A
:102770000D928A95E1F7812F2796EAE00C94552473
:102780000F931F93CF93DF93EC018B0145E453E14B
:102790000E941213882331F044ED52E1B801CE01BA
:1027A0000E941213DF91CF911F910F9108950F9303
:1027B0001F93CF93DF93C091A801D091A901CE01BF
:1027C000019626E0FB01DC0101900D922A95E1F7CC
:1027D00066E070E00E94AD1688836F8178858985F8
:1027E0009A8500915A0210915B0220915C0230910F
:1027F0005D02601771078207930751F060935A02D8
:1028000070935B0280935C0290935D020E941410AF
:10281000DF91CF911F910F9108950E94DB1E0E94BE
:102820007A0D0E94E81E08950E94ED1E0E948B0DF5
:102830000E94071F08950E94971C0E94C11E0E94BB
:10284000620D0E940D140E9414140E94700DFBCFA3
:102850008091740280FF0DC060911F0170E0660FCF
:10286000771F6038710570F56115710569F1862F64
:10287000089581FF07C060911F0184E0689FB00147
:102880001124EFCF60911F0182FD0AC08091730275
:102890008823A9F020911E0160911F01821710F07A
:1028A00088E0ECCF869FC001112433E0880F991F88
:1028B0003A95E1F7622F70E00E941724D2CF68E0CA
:1028C00070E0D5CF8FE7089581E00895809174027C
:1028D00080FF0CC060911C0170E07595679575953F
:1028E00067956115710549F1862F089581FF06C02E
:1028F00060911C0170E075956795F3CF60911C01A4
:1029000082FD0BC0909172029923A1F060911B018E
:1029100080911C01961738F0682F70E060387105BF
:1029200000F38FE70895899FC001112470E00E9491
:102930001724F4CF61E070E0D7CF81E008958D3C9B
:1029400031F40E94281481958093780208958E3C7A
:1029500019F40E942814F8CF8F3C31F40E942814F7
:102960008195809377020895803D19F40E94281480
:10297000F8CF893D29F40E94661480937902089566
:102980008A3D21F40E9466148195F7CF8B3D31F486
:102990000E946614819580937A0208958C3D19F403
:1029A0000E946614F8CF9FE2980F983070F4815D12
:1029B000990B21E030E001C0220F8A95EAF780915F
:1029C0007602822B8093760208958D3D31F48091BA
:1029D000740281608093740208958E3D21F4809189
:1029E00074028260F7CF8F3DB9F7809174028460E2
:1029F000F1CF409177028D3C59F48091780287FFA6
:102A00000DC01092780241110BC01092730208C0E1
:102A10008E3C81F48091780218169CF3442381F057
:102A20008091790290917A02892B09F05AC0109214
:102A3000720208958F3C49F447FFF0CF109277025D
:102A4000809178028111ECCFE0CF803D19F414160B
:102A5000ACF3E4CF90917902893D29F41916F4F68C
:102A600010927902DBCF8A3D19F497FFD7CFF8CFC8
:102A700090917A028B3D29F497FFD0CF10927A0281
:102A8000CDCF8C3D19F41916CCF3C8CF9FE2980F27
:102A9000983090F4815D990B21E030E0B90102C0DB
:102AA000660F771F8A95E2F7CB01809590917602A9
:102AB000892380937602B2CF8D3D31F480917402E8
:102AC0008E7F80937402AACF8E3D21F48091740290
:102AD0008D7FF7CF8F3D09F0A1CF809174028B7F5E
:102AE000F0CF08950E94FE1C9C0190917702809186
:102AF0007802982B21F0309371022093700290910C
:102B0000790280917A02982B21F030936F02209302
:102B10006E0285E792E00E94A21B089586E0E5E739
:102B2000F2E0DF011D928A95E9F71092730210928C
:102B30007202109274020895FC01828181110EC00C
:102B4000838181110BC08481811108C091E085814E
:102B5000811101C090E0892F8170089581E0FCCF40
:102B6000A6E0B0E0E6EBF5E10C94402486E0E5E772
:102B7000F2E0DE01119601900D928A95E1F7109234
:102B80007702109278021092790210927A028B8169
:102B90009C81892B89F080917002909171020E9432
:102BA000161DAC01909173029923C9F18091200107
:102BB0008417150608F440C08D819E81892B91F001
:102BC00080916E0290916F020E94161DAC0190914F
:102BD0007202992309F471C080911D0184171506B2
:102BE00008F479C0BE016F5F7F4F85E792E00E94D5
:102BF0004F1C811105C085E792E00E949C15811150
:102C00000E94721586E0FE013196A5E7B2E00190C0
:102C10000D928A95E1F72696E3E00C945C242091CE
:102C20006D028AE0289F900111242417350720F6B1
:102C30009F5F9093730202C09F3FD1F71B811123C6
:102C400059F00E9428149FEF11160CF491E0899F0F
:102C5000802D1124809377021C81112359F00E944A
:102C600028149FEF11160CF491E0899F802D1124F8
:102C70008093780230917702332309F49DCF20911D
:102C80007802222309F498CF45EB3403C0011124C4
:102C9000992359F09093770245EB24039001112476
:102CA000332339F03093780287CF81E08093770225
:102CB000F3CF81E0809378027FCF20916C028AE08D
:102CC000289F900111242417350708F08BCF9F5FB0
:102CD0009093720202C09F3FD1F71D81112359F0DA
:102CE0000E9466149FEF11160CF491E0899F802DCD
:102CF0001124809379021E81112359F00E946614D9
:102D00009FEF11160CF491E0899F802D1124809380
:102D10007A0230917902332309F464CF20917A0248
:102D2000222309F45FCF45EB3403C001112499231A
:102D300059F09093790245EB240390011124332339
:102D400039F030937A024ECF81E080937902F3CF4D
:102D500081E080937A0246CF0895FC01680F791FC5
:102D60008FEF91E3E617F70709F408952191822781
:102D700028E030E087FF06C0880F892721503109FD
:102D8000C9F7F0CF880FFACFCF93DF93EC01FB01A7
:102D90008581882309F4D2C09E0130572332310542
:102DA00008F0B2C00E948E0C90939B0280939A020E
:102DB000FE01E150F047E232F10520F4EE50FB4D08
:102DC0000C942B2480919A02816080939A0293C084
:102DD00080919B02886080939B028DC080919A02B3
:102DE0008260F3CF80919A028460EFCF80919A0243
:102DF0008860EBCF80919B028160EDCF80919B0238
:102E00008260E9CF80919A028061DFCF80919A023F
:102E10008062DBCF80919A028064D7CF0E94D40673
:102E200080919A028068D1CF80919A028C60CDCF38
:102E300080919B028360CFCF80919A028E7FC5CF15
:102E400080919B02877FC7CF80919A028D7FBDCFF3
:102E500080919A028B7FB9CF80919A02877FB5CFFC
:102E600080919B028E7FB7CF80919B028D7FB3CFE5
:102E700080919A028F7EA9CF80919A028F7DA5CFF3
:102E800080919A028F7BA1CF0E94D40680919A02F2
:102E90008F779BCF80919A02837F97CF80919B02FF
:102EA0008C7F99CF80919A0282FB992790F921E03B
:102EB000922790FB82F990FB83F987CF80919B0248
:102EC000982F909591708E7F892B90FB81F983CFFD
:102ED00090919A02892F8F7B96FF806476CF0E9413
:102EE000D40690919A02892F97FB87F980586DCF6D
:102EF00081E00E941A0D80919A0290919B020E949B
:102F0000930C0E94D40680E0DF91CF91089580E079
:102F1000F0CF90919A02892F8F7E94FF806155CFD8
:102F200090919A02892F8E7F90FF81604ECF909171
:102F30009B02892F877F93FF88604DCF81E0E4CF8C
:102F40008B3109F465C040F58B3071F078F4863030
:102F500009F447C020F4853059F180E008958730A6
:102F600009F448C08830C9F781E00895803109F438
:102F70005DC068F48E3089F790914602892F8B7F6F
:102F800092FF84608093460282FD4CC0EDCF863173
:102F900059F3893149F3E1CF8A3201F160F4873284
:102FA000B1F020F48E31C8F28D514CC08932A9F6AF
:102FB0000E948202D9CF833440F48A3308F041C0A2
:102FC000853329F0883381F2C8CF833431F681E02C
:102FD00090E00E9421070E94D406C6CF0E94170DE0
:102FE000C3CF80914602807F8093460281E0809328
:102FF0007E02089590914602892F8E7F90FF816016
:103000008093460280FDB0CF817F80934602ACCF93
:1030100090914602892F8D7F91FF826080934602B6
:1030200081FFA2CF809146028160EFCF909146024E
:10303000892F877F93FF88608093460283FDF2CFBC
:1030400093CF895321E030E0A90102C0440F551FFE
:103050008A95E2F7CA01BDCF80E008950E942C183E
:103060000895CF93C82F80917E028130B9F08823D4
:1030700031F08230A1F110927E0280E00DC00E94FA
:10308000780B8232D1F78C2F0E942C1881111BC033
:103090008C2F0E94A0178170CF9108950E94780B09
:1030A000823289F38C2F0E942E1881110AC0C431FC
:1030B00099F060F4CB3029F0C03169F782E0809359
:1030C0007E0281E0E8CF81E090E0E5CFC93221F0D7
:1030D000C833B9F380E0DFCF10927E02FBCFC93254
:1030E00009F43FC0E8F4C431E1F128F4C73009F431
:1030F0005BC081E0D1CF82EE8C0F8A30D0F7CD510A
:10310000C0937D02C33009F446C0B0F5C13009F464
:103110003FC080E291E0C230B1F110927D02E9CF70
:10312000C03509F452C0B8F48AE0CF3411F7E09109
:103130007B02F0917C023097E1F22081082E000C96
:10314000990B820F911D8F3F910509F00CF441C03E
:103150008FEF8083CECFC135D1F181E0C23539F315
:103160009BCF80917D02882321F210927D021092E4
:103170007C0210927B02BDCFC53099F078F08BE1D4
:1031800091E0C63051F690937C0280937B02B1CFE0
:103190008DE692E0F8CF8FE191E0F5CF8EE191E0FE
:1031A000F2CF8CE191E0EFCF10926D0284E1809339
:1031B0002001C0931F018CE380931E0188E080935F
:1031C0001C0188E280931B0194CF86EFB0CF8FEF74
:1031D000AECF97FFBECF10828CCFCF93DF93EB01A2
:1031E00086319C4711F50E94780B9D81992399F0B7
:1031F0008A7A91E009F490E090937F02811109C0EE
:1032000089E20E94500B0E94D10B80E0DF91CF91A8
:10321000089585E3F6CF80917F02811104C089E291
:103220000E94580BF0CF85E3FBCF81E0EFCF0F93E7
:103230001F93CF93DF93C42FD22FFC018581882366
:10324000C9F0409382020E94FE1C909381028093F9
:10325000800280E28C0F883040F4C77081E001C0AA
:10326000880FCA95EAF70E948004DF91CF911F91E1
:103270000F91089510918202141332C08091800240
:10328000909181020E94161D883C910548F5C0E28C
:10329000CD0F1D17B9F080E2810F883040F4177010
:1032A00081E001C0880F1A95EAF70E948704C830B0
:1032B00048F481E09D2F977001C0880F9A95EAF736
:1032C0000E948004802F0E947704C83070F6D77067
:1032D00081E001C0880FDA95EAF70E948704C5CF24
:1032E00080E28C0F883008F6C77081E001C0880F3B
:1032F000CA95EAF7F2CF0F93DB0188519C478730DC
:103300009105A0F5FC01EC5EFA4D0C942B2406E22D
:1033100021EE41EE6AE17CE7CD010E94171980E0C1
:103320000F91089507E225EE45EE6BE17CE7F4CFBF
:1033300006E221EE40EE68E17CE7EECF07E225EE03
:1033400044EE69E17CE7E8CF06E221EE42EE6CE173
:103350007CE7E2CF07E225EE46EE6DE17CE7DCCFCD
:1033600008E221E045EE6EE17CE7D6CF15968C9120
:10337000882319F010928202D3CF81E0D1CF8EE161
:10338000489B02C08150E1F7489BFECF08955898B2
:1033900080E28A95F1F7589A0895FC013BE03A954E
:1033A000F1F798E020E080E031E040E14A95F1F764
:1033B000880F489B02C08160232742E04A95F1F7BD
:1033C000000040E14A95F1F7915079F790E19A9524
:1033D000F1F799B132E03A95F1F7000040E14A95F2
:1033E000F1F7917092272081920F90830895A1E0C8
:1033F000B0E0EDEFF9E10C943D2419828C017C01E1
:10340000E60EF11C0E151F0541F481E09981911122
:1034100080E02196E6E00C9459240E94BF19CE0169
:1034200001960E94CD19F80181938F01EBCF509A3C
:10343000589A08955098589AE89AE9E6F0E0808101
:103440008C7F808308956150770B91E001C0990FC4
:103450006A95EAF720E031E0911108C0222391F04B
:10346000589A80E28A95F1F758980895492F482391
:1034700039F0589A232740E24A95F1F79695ECCF18
:103480005898F9CF5898EDCFFF920F931F93CF9391
:10349000DF93EC018C01060F111DC017D10729F431
:1034A000CDB7DEB7E5E00C945A24F9900E94C71915
:1034B00068E08F2D0E94231AF0CF1F920F920FB653
:1034C0000F9211240F931F932F933F934F935F936A
:1034D0006F937F938F939F93AF93BF93EF93FF93DC
:1034E000CF93DF930F92CDB7DEB719820E94BF1939
:1034F000CE0101960E94CD19082F069506950695D6
:10350000282F22952570902F9570290F922F937058
:1035100026952695920F982797708981982B09F008
:103520005CC0043008F059C080E18A95F1F7589AE0
:10353000509A82E08A95F1F700C0589888E0089F79
:1035400080011124D801AD5FBE4F1696ED91FC911C
:1035500017973097A9F06091A8017091A90114966E
:103560002D913C911597260F371F11968D919C91A7
:103570001297680F791F13964C9113978C910995A8
:10358000F801ED5FFE4F6381662351F02091A801A1
:103590003091A90184819581820F931F0E94441A62
:1035A0000E94C71980E18A95F1F758985098589A67
:1035B00080E18A95F1F7F801ED5FFE4F60816623A7
:1035C00051F02091A8013091A90181819281820F4F
:1035D000931F0E94F7190E94BF190F90DF91CF919E
:1035E000FF91EF91BF91AF919F918F917F916F91DB
:1035F0005F914F913F912F911F910F910F900FBEAF
:103600000F901F9018950F931F93CF93DF93EC01AA
:1036100004970CF04CC0F894509A589885E08A951D
:10362000F1F700009C2F969595708C2F8570980F60
:10363000892F83709695969523E0CC0FDD1F2A95F0
:10364000E1F7980F8E01092B0E94C71900C068E0AE
:10365000802F0E94231A80E18A95F1F75098589A9A
:10366000489B1EC087E090E048991CC0FE01ED5FBA
:10367000FE4F63816623F9F02091A8013091A901E2
:1036800084819581820F931F0E94F719811113C0C5
:10369000509A589A7894DF91CF911F910F91089585
:1036A00000C0DECF019729F4509A589A789480E0B0
:1036B000F2CF00C0D9CF0E94BF1980E28A95F1F7FE
:1036C0005898509A80E18A95F1F7CD5FDE4F688176
:1036D000662351F02091A8013091A90189819A8136
:1036E000820F931F0E94441A0E94C719789481E0A8
:1036F000D2CF9093AB018093AA0108959093890251
:103700008093880208950E941712811103C080914E
:1037100083020895E0918802F0918902309729F0A0
:103720000190F081E02D0995089580E00895E091E1
:103730008802F0918902309721F00280F381E02D18
:1037400009950895E0918802F0918902309739F047
:1037500022E0DC012C930480F581E02D0995089589
:10376000A3E0B0E0E6EBFBE10C944124209186025B
:103770003091870228173907A1F090938702809330
:103780008602E0918802F0918902309751F023E09F
:1037900029839B838A830680F781E02DCE010196E1
:1037A00009952396E2E00C945D24A3E0B0E0EBEDF4
:1037B000FBE10C944124209184023091850228176A
:1037C0003907A1F09093850280938402E0918802EA
:1037D000F0918902309751F024E029839B838A83FA
:1037E0000680F781E02DCE01019609952396E2E04F
:1037F0000C945D249C012E5F3F4FAC01485F5F4FEE
:1038000080E02417350709F40895F90191919F018B
:103810009923B9F38F5FF5CF662349F0FC01329607
:1038200008962191261729F0E817F907D1F780E0CB
:10383000089581E008959C01FC0132969FEF80E09D
:103840004191461751F09F3F19F4411101C0982F43
:103850008F5F8630A9F79F3F09F40895290F311D26
:1038600097FD3A95F90162830895FC013296089616
:103870002191261303C0DF0111971C92E817F90765
:10388000B9F708950E941B1C08950E94351C0895E5
:10389000029626E0FC0111922A95E9F7089546E088
:1038A00050E00E947C2421E0892B09F420E0822F43
:1038B000089508950E94591C0895811106C081E061
:1038C00080938A020E945A1C089582E0F9CF83E017
:1038D00080938A020E945A1C08950E945D1C0895DC
:1038E00081E080938A020E945A1C08950E94701CF5
:1038F0000895089508950E947A1C089508950895E2
:103900000E94791C0895CF930E947E1C0E949B11F7
:103910000E947F1CC0E08C2F0E947410811105C092
:10392000CF5FCC30C1F7CF91089581E0FCCF85B750
:10393000806885BF85B7806885BF08951F921FB6D0
:103940001F9211248F939F93AF93BF9380918B020B
:10395000811113C08091B6029091B702A091B80274
:10396000B091B9024196A11DB11D8093B60290930A
:10397000B702A093B802B093B902BF91AF919F91E3
:103980008F911F901FBE1F9018958091BE028430AA
:1039900031F10E94E20210928B0288E190E020E473
:1039A0000FB6F894A895809360000FBE2093600036
:1039B00083B7817F846083BF83B7816083BF78943E
:1039C000889583B78E7F83BF0FB6F894A8958091B2
:1039D0006000886180936000109260000FBE0895BF
:1039E0000E94D4060E94E702089582E084BD93E01D
:1039F00095BD9AEF97BD80936E0008952FB7F89408
:103A00008091B6029091B702A091B802B091B9022C
:103A10002FBF08952FB7F8946091B6027091B70246
:103A20008091B8029091B9022FBF08959C014FB7C1
:103A3000F8948091B6029091B702A091B802B0912B
:103A4000B9024FBF821B930B0895CF92DF92EF9282
:103A5000FF922FB7F894C090B602D090B702E090D2
:103A6000B802F090B9022FBFA7019601261B370BB1
:103A7000480B590BCA01B901FF90EF90DF90CF902E
:103A8000089578941F921FB61F9211248F939F93CD
:103A9000AF93BF938091B6029091B702A091B80204
:103AA000B091B9020196A11DB11D8093B602909309
:103AB000B702A093B802B093B902BF91AF919F91A2
:103AC0008F911F901FBE1F90189587E797E79093DF
:103AD00001088093000888E19AE00FB6F894A89551
:103AE000809360000FBE90936000FFCF88E19AE062
:103AF0000FB6F894A895809360000FBE9093600075
:103B0000FFCF8091940208959B01BA019091BE026B
:103B10009430E9F48F708093E9009FEF8091E80082
:103B2000915085FD06C085ED8A95F1F70000911151
:103B3000F5CF8091E80085FF0AC050E040E0C90160
:103B40000E947E1F8091E8008E778093E8000895A0
:103B500043E050E0BC0182E00E94841D089546E0ED
:103B600050E0BC0182E00E94841D0895CF93DF9352
:103B7000EC0148E050E0BC0181E00E94841D88E037
:103B8000FE01ACE8B2E001900D928A95E1F7DF9179
:103B9000CF9108958091BD02811109C00E940E212C
:103BA0000E946B218091E20084608093E20008957E
:103BB0001092BD0208950E94701C08956091BA028F
:103BC00081E0611101C080E00E94671C089590911E
:103BD000BE0281E0943009F080E06091BA020E9458
:103BE0006D1C089542E061EC81E00E948A2042E26F
:103BF00061EC82E00E948A209091BE0281E09430C4
:103C000009F080E06091BA020E945D1C08958091E5
:103C1000C002833009F461C030F48130D1F18230C8
:103C200009F49EC008958A3009F48AC08B3009F4E3
:103C30006FC0893009F050C08091BF02813209F015
:103C40004BC08091C3029091C402029708F044C017
:103C50008091E800877F8093E8008091E80082FFF0
:103C600037C09091F3008091F200029731F4809177
:103C7000F100813011F0863021F48091F1008093C1
:103C800094028091E8008B778093E8000E94BE2028
:103C900023C08091BF02813AF9F48091E800877FC8
:103CA0008093E8008091C3029091C402892B61F453
:103CB00068E08CE892E070E00E94CD1F8091E800FF
:103CC0008B778093E800089560E090E080E0F3CF88
:103CD0008091BE028111C1CF08958091BF02813AC7
:103CE000D9F78091C3029091C402892BA9F78091E2
:103CF000E800877F8093E8008091E80080FFFCCF98
:103D0000809129018093F1008091E8008E77BCCFEB
:103D10008091BF02813201F78091C3029091C40269
:103D2000892BD1F68091E800877F8093E8000E947C
:103D3000BE208091C102809329010E94D40608957B
:103D40008091BF02813241F68091E800877F8093A5
:103D5000E8000E94BE208091C202809395020895DF
:103D60008091BF02813A09F0B7CF8091E800877F48
:103D70008093E8008091E80080FFFCCF809195025D
:103D8000C1CF84B7877F84BF0FB6F894A895809180
:103D90006000886180936000109260000FBE80E830
:103DA00090E00FB6F89480936100909361000FBE8D
:103DB0000E94761C08950E940E210E946B21E2EE63
:103DC000F0E080818460808378940E94EA230895E3
:103DD00081E291E00E947E1B08958091BE028530B1
:103DE00031F48091BE02853019F00E94F01C0895D4
:103DF0000E94C51C8091BC02882399F30E94831CF9
:103E0000882379F30E94681F0E94D406EACF0895A0
:103E10009A014091C5025091C6020E94101F089558
:103E2000492F55274330510519F168F441305105A8
:103E300009F444C04230510509F445C090E080E0E7
:103E400050E040E025C04132510549F14232510570
:103E5000A9F780E490E046E653E061157105C1F0F2
:103E60008BE790E04BEE52E06130710589F0E6CFD0
:103E700099278130910581F0009729F00297F1F69A
:103E8000ECE5F2E002C0EAE9F2E0849190E0AF01F3
:103E9000F901518340830895EAE8F2E0F6CF89E022
:103EA00090E040EB52E06115710591F389E090E0FC
:103EB00049EC52E06130710559F3C0CF82E190E0E6
:103EC00049ED52E0E5CF8BE390E04EE952E0E0CFE0
:103ED00080E189BD82E189BD09B400FEFDCF8091FA
:103EE000D8008F7D8093D8008091E000826080931D
:103EF000E0008091E00081FDFCCF0895AF92BF9279
:103F0000CF92DF92FF920F931F93CF93DF936C01B9
:103F1000EB018A010E94DD20F82E811123C00115DA
:103F2000110539F0F80180819181C81BD90BC80EA9
:103F3000D91EB12CA12C2097A9F08091E80085FD15
:103F400022C08091E8008E778093E800011511056A
:103F5000A1F0F80180819181A80EB91EB182A082E2
:103F600085E0F82E8F2DDF91CF911F910F91FF905B
:103F7000DF90CF90BF90AF9008950E94DD208823FE
:103F8000D1F2F82EEFCFF60181916F018093F1000D
:103F90002197FFEFAF1ABF0ACECFFC018091C50277
:103FA0009091C60286179707A0F06115710529F454
:103FB0009091E8009E779093E80090E0611571057C
:103FC00051F4911108C08091E80082FF34C080E074
:103FD0000895BC01F2CF8091BE028823C1F18530E3
:103FE000C1F18091E80083FD30C08091E80082FD3E
:103FF000EACF8091E80080FFE1CF8091F30020912B
:10400000F200382F6115710519F02830310558F08C
:1040100091E02830310509F090E02091E8002E77FA
:104020002093E800CBCF81918093F100615071091A
:104030002F5F3F4FE7CF8091BE02882341F085304C
:1040400041F08091E80083FFBECF81E0089582E0D7
:10405000089583E00895FC018091C5029091C60205
:1040600086179707A0F06115710529F48091E80083
:104070008E778093E80090E06115710551F49111FD
:1040800008C08091E80082FF35C080E00895BC013F
:10409000F2CF8091BE028823C9F18530C9F18091A9
:1040A000E80083FD31C08091E80082FDEACF809175
:1040B000E80080FFE1CF8091F3002091F200382FDB
:1040C0006115710519F02830310558F091E028305C
:1040D000310509F090E08091E8008E778093E80048
:1040E000CBCF84918093F1003196615071092F5F9D
:1040F0003F4FE6CF8091BE02882341F0853041F0EA
:104100008091E80083FFBDCF81E0089582E00895AB
:1041100083E00895982F973028F08F708093E900FE
:1041200081E008959093E900242F762F50E09817AE
:1041300031F07091EC002091ED005091F00021FDE4
:1041400002C09F5FE8CF3091EB003E7F3093EB00E1
:104150003091ED003D7F3093ED003091EB00316008
:104160003093EB007093EC002093ED005093F0003F
:104170002091EE0027FDE5CF80E008958091BF02F9
:1041800087FF13C08091E80082FF06C08091E8009D
:104190008B778093E80004C08091BE028111F2CF3A
:1041A00008958091BE028823D9F38091E80080FFB2
:1041B000F8CF8091E8008E77ECCF2091E400309129
:1041C000E50095E6A9012091EC00822F817020FF87
:1041D00006C08091E80080FF06C080E0089520912D
:1041E000E80022FD1AC08091BE02882389F0853044
:1041F00089F08091EB0085FD0FC02091E4003091A3
:10420000E50042175307F9F29150E1F684E0089572
:1042100082E0089583E0089581E008950E947D2161
:104220000E948521E0EEF0E0808181608083E8EDEE
:10423000F0E080818F77808319BCA7EDB0E08C918E
:104240008E7F8C9380818F7E80831092BD02089533
:104250000F931F93CF93DF930E947D210E948521AE
:10426000C8EDD0E088818F778883888180688883D3
:1042700088818F7D888319BC1092BE021092BA0289
:104280001092BC021092BB0200EE10E0F801808197
:104290008B7F808388818160888342E060E080E05A
:1042A0000E948A20E1EEF0E080818E7F8083E2EE42
:1042B000F0E0808181608083808188608083F80164
:1042C00080818E7F8083888180618883DF91CF9118
:1042D0001F910F910895E8EDF0E080818F7E80833B
:1042E000E7EDF0E080818160808384E082BF81E03F
:1042F0008093BD020E9428210895E8EDF0E08081BE
:104300008E7F80831092E20008951092DA0010925E
:10431000E10008951F920F920FB60F9211242F9370
:104320003F934F935F936F937F938F939F93AF933D
:10433000BF93EF93FF938091E10082FF0BC08091C8
:10434000E20082FF07C08091E1008B7F8093E10053
:104350000E94E9238091DA0080FF19C08091D80083
:1043600080FF15C08091DA008E7F8093DA00809103
:10437000D90080FF96C080E189BD82E189BD09B482
:1043800000FEFDCF81E08093BE020E94CA1D809195
:10439000E10080FF19C08091E20080FF15C080918C
:1043A000E2008E7F8093E2008091E2008061809342
:1043B000E2008091D80080628093D80019BC85E02B
:1043C0008093BE020E94DE1D8091E10084FF2BC01D
:1043D0008091E20084FF27C080E189BD82E189BD30
:1043E00089B5982F917080FFFBCF8091D8008F7D89
:1043F0008093D8008091E1008F7E8093E1008091CE
:10440000E2008F7E8093E2008091E20081608093E1
:10441000E2008091BA02882309F449C084E08093C5
:10442000BE020E94E71D8091E10083FF29C08091B8
:10443000E20083FF25C08091E100877F8093E10047
:1044400082E08093BE021092BA028091E1008E7FDA
:104450008093E1008091E2008E7F8093E200809162
:10446000E20080618093E20042E060E080E00E9430
:104470008A208091F00088608093F0000E94DB1D0C
:10448000FF91EF91BF91AF919F918F917F916F912C
:104490005F914F913F912F910F900FBE0F901F9002
:1044A000189519BC1092BE020E94D81D70CF809141
:1044B000E30087FD93E09093BE02B3CF1F920F926B
:1044C0000FB60F9211242F933F934F935F936F93E7
:1044D0007F938F939F93AF93BF93CF93DF93EF938C
:1044E000FF93D091E900DF708091EC00C82FC1707C
:1044F00080FDC0E81092E9008091F000877F8093F2
:10450000F00078940E94A2221092E9008091F000BD
:1045100088608093F000CD2BCF70C093E900FF91AD
:10452000EF91DF91CF91BF91AF919F918F917F914B
:104530006F915F914F913F912F910F900FBE0F9010
:104540001F901895AAE2B0E0E8EAF2E20C94402449
:104550008FEB92E02091F100FC012193CF01F2E07A
:10456000873C9F07B9F70E94071E8091E80083FFF0
:104570001EC18091BF029091C0029A3008F017C10D
:10458000E92FF0E0E55EFA4D0C942B24803899F089
:10459000823809F00CC18091C3028F70873008F017
:1045A00006C18093E9008091EB0085FB882780F9A4
:1045B0001092E90006C08091BB029091BC0291115B
:1045C00082609091E800977F9093E8008093F100DB
:1045D0001092F1008091E8008E77E5C0882309F4FD
:1045E000D3C0823009F0E3C08091C1028111D6C0EE
:1045F0008091C3028F702FEF280F263008F0D7C0AC
:104600008093E9002091EB0020FFC8C0933031F483
:104610008091EB0080628093EB00C0C09091EB0032
:1046200090619093EB0021E030E001C0220F8A9569
:10463000EAF72093EA001092EA008091EB0088608C
:10464000EACF8111B4C01091C1021F778091E300BD
:104650008078812B8093E3008091E800877F8093AE
:10466000E8000E94BE208091E80080FFFCCF80918E
:10467000E30080688093E30082E0111183E080937F
:10468000BE0295C08058823008F091C08091C1026E
:104690009091C2028C3D23E09207A1F583E08A83CA
:1046A0008AE289834FB7F894DE01139620E03EE05A
:1046B00051E2E32FF0E050935700E49120FF03C054
:1046C000E295EF703F5FEF708E2F90E0EA30C0F020
:1046D000C7968D939D932F5F243159F74FBF8091DB
:1046E000E800877F8093E8006AE270E0CE010196DF
:1046F0000E94CD1F8091E8008B778093E80057C01F
:10470000C096E7CF6091C3027091C402AE014F5FC3
:104710005F4F0E94081FBC01892B09F448C090918B
:10472000E800977F9093E80089819A810E942B206E
:10473000E1CF8038E1F58091E800877F8093E80041
:104740008091BA028093F10045CF811130C09091E1
:10475000C102923060F58091E800877F8093E80085
:104760009093BA020E94BE208091BA02882311F071
:1047700084E005C08091E30087FDFACF81E080935B
:10478000BE020E94F21D13C08091C102813079F4F3
:1047900081E0933009F080E08093BC021092E90040
:1047A0008091E800877F8093E8000E94BE2080917E
:1047B000E80083FF0AC08091E800877F8093E800CB
:1047C0008091EB0080628093EB00AA96E3E00C946A
:1047D0005C240895CF938091BE028823A1F0C091FC
:1047E000E900CF709091EC00892F817090FD80E8F6
:1047F000C82B1092E9008091E80083FD0E94A2225C
:10480000CF70C093E900CF9108950E940E211092BD
:10481000BE020895E8EDF0E08081806180838AE146
:104820008A95F1F700C08091D9008170089597FBB7
:10483000072E16F4009407D077FD09D00E94682453
:1048400007FC05D03EF4909581959F4F0895709593
:1048500061957F4F0895EE0FFF1F0590F491E02DB5
:1048600009942F923F924F925F926F927F928F9214
:104870009F92AF92BF92CF92DF92EF92FF920F93EF
:104880001F93CF93DF93CDB7DEB7CA1BDB0B0FB6F9
:10489000F894DEBF0FBECDBF09942A8839884888B6
:1048A0005F846E847D848C849B84AA84B984C8844C
:1048B000DF80EE80FD800C811B81AA81B981CE0F43
:1048C000D11D0FB6F894DEBF0FBECDBFED01089528
:1048D000AA1BBB1B51E107C0AA1FBB1FA617B70726
:1048E00010F0A61BB70B881F991F5A95A9F7809542
:1048F0009095BC01CD010895FB01DC0104C08D91B0
:104900000190801921F441505040C8F7881B990B41
:104910000895FB01DC0102C001900D92415050400E
:10492000D8F70895F999FECF92BD81BDF89A9927DD
:1049300080B50895A8E1B0E042E050E00C94D624A0
:10494000DC01A40FB51F4150504048F0CB01840F4B
:10495000951F2E910E94B12441505040D0F70895E8
:10496000262FF999FECF92BD81BDF89A019700B428
:10497000021639F01FBA20BD0FB6F894FA9AF99AC8
:104980000FBE08950396272F0E94B1240E94B024E1
:10499000252F0E94B124242F0C94B1240196272F97
:1049A0000E94B1240C94B024DC01CB01FC01F999E4
:1049B000FECF06C0F2BDE1BDF89A319600B40D926B
:1049C00041505040B8F70895F894FFCFCD04CD047E
:1049D0001D051D0582059E05FC04FC04A3051406A7
:1049E000230623061C1790172417EE16F216281715
:1049F000F6162C1738170217891706173C170A17CF
:104A0000401768170E1744176F1714174A175217D5
:104A1000FA163017FE16341718174E175E17781748
:104A20008717E8162017971798199E198719921952
:104A3000A419AA19B019C622EE22D723EE22D72331
:0A4A400021234223D7239923A52345
:104A4A00260201000000010000000000000006012B
:104A5A0000000004070000000000002808503C077E
:104A6A0014811DB61DAF1DA81D01E200E900EA0070
:104A7A00B500B600B700CD008301CC008A019201CF
:104A8A0094012102230224022502260227022A0275
:104A9A00B300B4006F0070009F01CB019F02A00217
:104AAA00818283E200E900EA00B500B600B700CDD2
:104ABA00008301CC008A019201940121022302247D
:104ACA00022502260227022A02B300B4006F0070F0
:104ADA00009F01CB019F02A002818283946697C640
:0A4AEA003435F6F7313332364F024F
:00000001FF
